:020000040000FA
:020000000728CF
:08000800AD0A0B1109000313FE
:1000100083120230850007309900A0308B00003039
:1000200083168C00C5308100083085008312203093
:1000300084008001840A041F19280030AB001622B6
:100040002130D423AE002430D423B1002230D42375
:10005000B800B3000230D423BE001E30D423C00049
:100060002330D423AC00AC182C150430B5003C125E
:100070000513E6213F205C20FD2024223A28203071
:10008000B9001330A900083005052A0603194E28C7
:10009000C320B90B51280830AA063F282A30A900EE
:1000A0004828C320083005052A0603194128C32023
:1000B000DF20A90B512808002508A1002608A2006E
:1000C0002708A3002808A400A501A601A701A801EC
:1000D000253084006E2076207E2008000830A9009C
:1000E000A120A420800DA90B7028C328840AA12078
:1000F000A420800DA120A420800DC328840A0430F0
:10010000A900A120A420800C840AA120A420800C96
:10011000A90303198D2884038128800E8403800E8F
:10012000C328083005052A060319B90A0800AA1DC4
:100130009D28C320851D99280800C32085199D2866
:100140000800AA199D289928AD01C320083005058B
:100150002A060319AE28AD18BC28A528C320C32041
:10016000C320B9019120C320C3209120C320DF20E8
:1001700091200230390208002030C2002F08C1004F
:10018000BE23972020282B18D2280512010C7F3976
:100190000319CE282F02031C05100800AF08031D09
:1001A000051408000510010C7F390319DB282F0204
:1001B000031C05120800AF08031D05160800BC1C2F
:1001C000FA2832082F02031CF82803103B0D2C1CC0
:1001D0003B08323E2C180A3EA000010CA002031876
:1001E000C3287D3C031CF6288513C3288517C32824
:1001F0008517C328AC188513C32821082502031DC1
:100200001D2922082602031D1D2923082702031D7C
:100210001D2924082802031D1D2921082E02031967
:1002200017292C1F1D2921083102031D1D29C32058
:10023000230824020319AA291E2908003C162808AD
:10024000FE3E03194529FF3E03198512FF3E03199F
:100250000513FF3E03194B29FF3E03199621FF3E6C
:1002600003197B21FD3E03195029FF3E0319851612
:10027000FF3E03190517FF3E03194829FF3E0319E6
:10028000A021FF3E03198921C4292308073C6F29B7
:100290002308F83E6F292308073C031863296F29B8
:1002A00008302702031C6F2903191D29FD3E03197D
:1002B0008516FF3E03190517FE3E0319A021FF3ED8
:1002C00003198921C42903197B21FF3E03199621B3
:1002D000FE3E03190513FF3E03198512C4292408A5
:1002E00001392B060319C42924080139AB001E2249
:1002F0000130A300C429AC1E8729BC1E0800B90028
:100300002230D423B800B300BC123908080085138A
:100310000800AC1E9429BC1A0800B9000130B800CE
:10032000B300BC1639080800851708002C1D9E294B
:10033000AC1C9C29BC1008003C11080005130800E7
:100340002C1DA829AC1CA629BC1408003C150800CB
:1003500005170800C3202308013A031DBF293C18D4
:10036000B529FF30B4000430B5003C186A223C18AF
:10037000C4293C14AB090130AB051E22C429AC18BA
:10038000BC143C1CC4293C10C320E6212308013ABC
:100390000319E3292308BB003C19DB290310BB0D1B
:1003A000AC1FDF29A2080319DF29221CBB0AA218EF
:1003B000DF29BB0ADF293C1EDF293030BB073B08A1
:1003C000D423B2000800B201AF0108002C1A082A99
:1003D0002B18F92985100515AF0803190511AC1D57
:1003E00005153C1A0800A218F72985120800851681
:1003F000080005118514AF0803198510AC1D85147C
:100400003C1A0800A218062A051308000517080060
:100410002B18102A8510A2180515A21C051108001A
:100420000511A2188514A21C851008002030D423C1
:10043000AF00B2002530D423AB0008002530C20045
:100440002B08C100BE2308003808013C031D2B2ADD
:100450003208AF00C3283C1232082F020319C32808
:10046000B30BC3283E082F0203183F2AB208031912
:100470003C2A3E08AF003F2AAF01B30AC328320826
:100480002F02031C452AAF03462AAF0A3808B300DF
:10049000AD012630D423C3202F08BF00C10B512A41
:1004A000552ABF070318AD0A4E2A0430C100C320E5
:1004B000AD0CBF0CAD13C10B572AAD080318622A4F
:1004C000AD0CBF0C2730D4233F084102031C003081
:1004D000B307C328B40B08006E2A0800FF30B4002D
:1004E000B50B0800A42AB600B60A0B30BC1BDA2BE9
:1004F000B60B7B2A080005158514DA230511851033
:10050000DA23782A0230B6002F30762A9122230887
:10051000013A0319862A91222308013A031D8B2AE6
:1005200008003F205C2021082502031D912A220893
:100530002602031D912A23082702031D912A24085D
:100540002802031D912A0800BC10093073220130D3
:1005500073228622E023B9030319D52AB9030319AC
:10056000DD2AB9030319E82AB9030319222BB903B9
:100570000319382BB90303194A2BB9030319522B5A
:10058000B9030319642BB9030319772BB9030319B2
:10059000892BB90303199C2B0430B9020319AA2B28
:1005A00021080319B62B8222A92A73228622213020
:1005B000C2002108C100BE23A72A7322862222304E
:1005C000C200E0233908C1002230C200BE23A72A9E
:1005D00073228622E023C2000310C20D21080319F2
:1005E000072B10303902031CF72A8222E92A390826
:1005F00073228622E0230310B90DB91F012B82223A
:10060000F92A3908C100BE2301307322E92A0630D5
:10061000B600D423B900B6033603D423B9020310BD
:10062000390CC1073608C200BE2383169C18162B4E
:100630008312B60A1E3036020318A72AB60AB60A73
:100640003608092B73228622E02304303902031C6A
:100650002B2B8222232B2330D423E730C105B9036F
:100660003918C115B91841162330C200BE23A72A74
:1006700073228622E02303303902031C412B82229D
:10068000392B2330D423C112391CC1162330C200A8
:10069000BE23A72A732286222430C2002108C1006B
:1006A000BE23A72A73228622E02303303902031CCB
:1006B0005B2B8222532B2330D4234113391C411747
:1006C0002330C200BE23A72A73228622E0230530EE
:1006D0003902031C6D2B8222652B2330D423F83082
:1006E000C1053908C1042330C200BE23A72A7322E2
:1006F0008622E02303303902031C802B8222782BD0
:100700002330D423C113391CC1172330C200BE23A8
:10071000A72A73228622E02304303902031C942B7B
:1007200021303902031C962B82228A2B2630C200EC
:100730003908C100BE23A72A73228622E023B90804
:10074000031DA42B82229D2B2730C2003908C10033
:10075000BE23A72A8622E02303303902031CB22BD2
:100760008222AA2BBC13391CBC17A72AFF30B40065
:100770000430B500013073228E21202841088316F1
:100780009A008312420883169B008B131C129C1143
:100790001C1555309D00AA309D009C141C119C18FE
:1007A000CF2B83128B17080083169B001C141A088A
:1007B00083120800AD01AD02AD08031DDC2B08005B
:1007C000B901A11FE62BB90A211FB90AA11EEC2B02
:1007D0000330B907211EB907A11DF22B0930B90753
:1007E000211DB907A11CF82B1B30B907211CB90723
:0407F00039080800BC
:02400E00C401EB
:104200000000000012000000140015001600180045
:104210001A001C001E0020002200250028002B0090
:104220002E00320036003A003E00430048004E00A7
:1042300054005A00600067006E0075007C000000AA
:1042400000002A000100A0002A00000010001E004B
:10425000000000000000000000000000000000005E
:104260000000000008000A000C000E001000120000
:10427000150018001B001E002100250029002D003C
:10428000FF00FF00FF00FF00FF00FF00FF00FF0036
:10429000FF00FF00FF00FF00FF00FF00FF00FF0026
:1042A000FF00FF00FF00FF00FF00FF00FF00FF0016
:1042B000FF00FF00FF00FF00FF00FF00FF00FF0006
:1042C000FF00FF00FF00FF00FF00FF00FF00FF00F6
:1042D000FF00FF00FF00FF00FF00FF00FF00FF00E6
:1042E000FF00FF00FF00FF00FF00FF00FF00FF00D6
:1042F000FF00FF00FF00FF00FF00FF00FF00FF00C6
:00000001FF
